:020000040000FA
:0C08000012EEFEF05CEF0AF016EF0AF0BA
:0408180039EF0AF0BA
:10082000010E0001646F0B0E0001665DD8B05AD056
:10083000FA6AFB6A6635FA36E834FA36FC0B4E0F74
:10084000E56E080EFA22000EFB22E450F96E3DEF31
:1008500004F041EF04F045EF04F049EF04F04DEFF0
:1008600004F051EF04F055EF04F059EF04F05DEFA0
:1008700004F064EF04F06BEF04F0010E0001636F0D
:1008800037D0010E0001636F33D0010E0001636F9A
:100890002FD0060E0001636F2BD00D0E0001636F89
:1008A00027D01D0E0001636F23D04C0E0001636F33
:1008B0001FD09A0E0001636F1BD09A0E0001636F68
:1008C000020E0001646F14D09A0E0001636F050ED2
:1008D0000001646F0DD09A0E0001636F0A0E0001D3
:1008E000646F06D09A0E0001636F140E0001646FEE
:1008F0000001606B00016751800A01E139D0800E70
:100900000001675D1BE28150675D0AE364C062F02D
:1009100063C061F0612FFED7622FFAD7602FF3D743
:100920008150675D0AE264C062F063C061F0612FCC
:10093000FED7622FFAD7602FF3D71AD08150675DA8
:100940000AE264C062F063C061F0612FFED7622FDB
:10095000FAD7602FF3D78150675D0AE364C062F075
:1009600063C061F0612FFED7622FFAD7602FF3D7F3
:100970000001606B080E0001665DD8B0F4EF06F070
:10098000FA6AFB6A6635FA36E834FA36FC0B9E0FD3
:10099000E56E090EFA22000EFB22E450F96EDFEF3D
:1009A00004F0E2EF06F0E9EF06F0E9EF06F0E9EF18
:1009B00006F0E9EF06F0E9EF06F0E9EF06F007EEE2
:1009C00000F081CFEEFF81CFEEFF81CFEEFF81CF30
:1009D000EEFF81CFEEFF81CFEEFF81CFEEFF81CF23
:1009E000EEFF81CFEEFF81CFEEFF81CFEEFF81CF13
:1009F000EEFF81CFEEFF81CFEEFF81CFEEFF81CF03
:100A0000EEFF81CFEEFF81CFEEFF81CFEEFF81CFF2
:100DC000EEFF20D007EE00F081CFEEFF602FFCD7C2
:100DD00019D007EE00F081CFEEFF63C061F0612F04
:100DE000FED7602FF8D70ED007EE00F081CFEEFFD0
:100DF00064C062F063C061F0612FFED7622FFAD742
:100E0000602FF4D7120000C0E5FF01C0E5FF02C06B
:100E1000E5FF0401196B1A6B04011151600BD8A492
:100E2000E6D012C400F00050050A0CE00050060A9B
:100E300011E00050080A01E1CCD00050090A01E19C
:100E4000B8D0D5D0040113510401276F040E04015A
:100E5000286FCAD014C400F0010E005CD8A0C7D01F
:100E6000040E005CD8B0C3D00006FA6AFB6A0034F6
:100E7000FA36E834FA36FC0B880FE56E0E0EFA22CD
:100E8000000EFB22E450F96E4AEF07F05CEF07F02A
:100E90006EEF07F0000E026E120E016E980E006EDD
:100EA000005004011C6F01501D6F02501E6F120E86
:100EB0000401196F1A6B79D0000E026E120E016ECA
:100EC000AA0E006E005004011C6F01501D6F0250ED
:100ED0001E6F200E0401196F1A6B67D013C400F047
:100EE000010E005CD8A050D0040E005CD8B04CD0ED
:100EF0000006FA6AFB6A0034FA36E834FA36FC0B6C
:100F0000100FE56E0F0EFA22000EFB22E450F96E70
:100F10008EEF07F0A0EF07F0B2EF07F0000E026EC1
:100F2000120E016ECE0E006E005004011C6F0150B7
:100F30001D6F02501E6F2C0E0401196F1A6B35D0F5
:100F4000000E026E120E016EFA0E006E00500401C9
:100F50001C6F01501D6F02501E6F220E0401196F8D
:100F60001A6B23D0000E026E130E016E1C0E006E63
:100F7000005004011C6F01501D6F02501E6F0C0EBB
:100F80000401196F1A6B11D0000E026E120E016E61
:100F9000CA0E006E005004011C6F01501D6F0250FC
:100FA0001E6F040E0401196F1A6B010E04011B6FF2
:100FB0001BD0040113510401296F295104E1050ECE
:100FC0000401286F11D0060E0401286FB0EC0AF05E
:100FD0000BD0290E04011C6F040E1D6F010E0401BD
:100FE000196F1A6B04011B6B94EC09F002D097EC9B
:100FF0000AF0E4CF02F0E4CF01F0E4CF00F01200F9
:1010000000C0E5FF01C0E5FF02C0E5FF03C0E5FF4A
:1010100004C0E5FF05C0E5FF06C0E5FF060E0401BC
:10102000285D02E36DA201D087D0040108BF84D0FF
:1010300000C600F0060E005CD8B063D0FA6AFB6A06
:101040000034FA36E834FA36FC0B5A0FE56E100E0F
:10105000FA22000EFB22E450F96E39EF08F041EF5E
:1010600008F049EF08F070EF08F079EF08F07DEF35
:1010700008F0020E006E010E0501006F010E016FF7
:1010800041D0010E006E10EC04F0010E0501006F5E
:1010900039D006010151400DF3CF01F0026A400E34
:1010A000025C1BE2000E0224036E046A050E042299
:1010B000000E0124056E066A070E062205C0E9FF30
:1010C00006C0EAFFEFCF05F003C0E9FF04C0EAFF66
:1010D00005C0EFFF022A012AE2D7400E006E12D0AF
:1010E0000F0E06010115016EC00E0110B56E006AEB
:1010F00009D001C666F0006A05D001C667F0006A33
:1011000001D0006A00500CE0005004010D6F040192
:101110000CAD03D0880E0C6F03D0C80E04010C6F09
:10112000400E0401096F040108AD03D0880E086F5A
:1011300003D0C80E0401086FE4CF06F0E4CF05F039
:10114000E4CF04F0E4CF03F0E4CF02F0E4CF01F009
:10115000E4CF00F0120000C0E5FF01C0E5FF02C0CF
:10116000E5FF000E04011A5D02E1080E195D04E2BC
:1011700004011951006E02D0080E006E00500401E7
:10118000056F00C001F0026A01500401195F0250AE
:101190001A5B04EE1FF004011B51010A17E11CC485
:1011A000F6FF1DC4F7FF1EC4F8FF00C001F0015098
:1011B00005E00900F5CFEEFF0106F9D7F65004016E
:1011C0001C6FF7501D6FF8501E6F0FD01CC4D9FF55
:1011D0001DC4DAFF005004E0DECFEEFF0006FAD7B0
:1011E000D95004011C6FDA501D6FE4CF02F0E4CF38
:1011F00001F0E4CF00F0120000C0E5FF01C0E5FF00
:101200006C5020E100C400F03C0E0014016E01504F
:10121000340A07E103EC07F0C80E0401046F6D986F
:1012200036D004011051020A0AE100AC04D0880E45
:101230000401006F2CD0C80E0401006F28D07DEC93
:101240000AF025D06C50040A22E104012851040A56
:101250000CE127C46EFF6E5005E0050E0401286FF7
:10126000808A03D0030E0401286F04011051010A83
:101270000CE1ABEC08F0040104AD03D0880E046F60
:1012800006D0C80E0401046F02D07DEC0AF0E4CF52
:1012900001F0E4CF00F0120012010002000000088B
:1012A000501D30600201010203010902200001010A
:1012B0000080FA0904000002000000000705010296
:1012C00040000007058102400000040309042C03CC
:1012D00049006C006C006500670061006C00200034
:1012E000530079007300740065006D0073002000E6
:1012F00043006F00720070002E002203490053006B
:10130000430020004F007300630069006C006C0014
:101310006F00730063006F00700065000C035600DF
:1013200031002E003000320000C0E5FF01C0E5FFB3
:10133000040111AF28D0010E0401106F17C400F092
:1013400018C401F004011A51015C02E11951005C5A
:1013500004E200C019F401C01AF4ABEC08F01F0E4F
:101360000401066F040E076F080E0401016F110ED1
:10137000006E040E016E0050026F0150036F800E6C
:101380000401006F0FD0020E0401106F080E04015B
:10139000016F1F0E026F040E036FC80E0401006F71
:1013A0000401056BE4CF01F0E4CF00F0120000C0AF
:1013B000E5FF01C0E5FF69506814006E00A405D088
:1013C0006D9269946894689869880050016E01A0D4
:1013D00012D068A602D06896FCD7686A7B0E696E48
:1013E0006E6A160E706E7DEC0AF06D980401296B22
:1013F000030E0401286F00A803D0698468986D82E9
:1014000000AA06D070A003D07DEC0AF07090689A14
:10141000030E0401285D05E300A603D0FCEC08F0F0
:101420006896E4CF01F0E4CF00F01200D8CFE5FFDA
:10143000E0CFE5FFE56EF3CFE5FFF4CFE5FFE9CFC1
:10144000E5FFEACFE5FFFACFE5FFFBCFE5FFE4CF0D
:10145000FBFFE4CFFAFFE4CFEAFFE4CFE9FFE4CFFC
:10146000F4FFE4CFF3FFE450E4CFE0FFE4CFD8FF94
:101470001000D8CFE5FFE0CFE5FFE56EF3CFE5FF45
:10148000F4CFE5FFE9CFE5FFEACFE5FFFACFE5FFCF
:10149000FBCFE5FFE4CFFBFFE4CFFAFFE4CFEAFFA9
:1014A000E4CFE9FFE4CFF4FFE4CFF3FFE450E4CF6F
:1014B000E0FFE4CFD8FF1000806A0F0E926E070E97
:1014C000B46EE70EB56E0F0EC16E816AFF0E936E9D
:1014D000826A3B0E946E1F0EBD6EBE6ACB6ACC6AEA
:1014E000040ECA6E010E0001666FC5EC0AF0D7EC5F
:1014F00009F000EC08F0FBD7120000C0E5FF01C0C6
:10150000E5FF0401106B080E0401016F110E006E5F
:10151000040E016E0050026F0150036F880E04012B
:10152000006F046BE4CF01F0E4CF00F0120000C0C4
:10153000E5FF01C0E5FF080E0401016F110E006E0A
:10154000040E016E0050026F0150036F840E0401FF
:10155000006F840E046FE4CF01F0E4CF00F01200BE
:101560001E0E716E400E0401096F000E0A6F060E0A
:101570000B6F880E0401086F000E04010E6F050E3C
:101580000F6F400E04010C6F12000401006B046B1E
:10159000140E6F6E080E6D6E6DBAFED7686A110E6E
:0A15A000696E020E0401286F1200AC
:020000040030CA
:0E000000E03EF8FEFF7D9AFFFFFFFFBFFFFF0F
:00000001FF
